:020000040000FA
:06000000653003303A28D0
:08000800A000030EA100831209
:100010008B1C32288B1031181428B11C3228643004
:10002000010203183128182800001628172818285C
:1000300019281A281B281C281D281E281F283110A3
:10004000B114A810031005190314AA0DA90DA80DC9
:10005000B00B322831152A08AF002908AE00280855
:10006000AD00B11081010B11210E8300A00E200EF6
:02007000090085
:0C007400203084008001840A6030040207
:10008000031C3C281230B000A0218316FF239000EF
:10009000831283160C308505870183128501870141
:1000A000073099000030831691009F008312C830FA
:1000B00083168100831231309000003083168C004B
:1000C000831210308B00302281018E018F010B11C1
:1000D0008B100B108C018B177B2031199120B30BE7
:1000E0007928031085190314B90DF030390203196A
:1000F000172131226C286400311808000B1D0800FC
:100100000B11B11031141230B000051D8C283214BF
:10011000831601138312080032108316011783120D
:10012000080031110130B70085148B1320303707D8
:1001300083169B001C141A088312A400A500C0306B
:10014000A5061030370783169B001C141A0883126B
:10015000A3000030370783169B001C141A08831273
:10016000A2008B17321CBA2822090339A200A30966
:10017000A409A50922082D02031D112923082E0216
:10018000031D112924082F02031DE2280130370224
:10019000031DCD283D143E14B52102303702031D46
:1001A000D428BD143E14BD2103303702031DDB28C3
:1001B0003D153E14C52104303702031DE228BD154C
:1001C0003E14CD2125082F02031D032901303702DB
:1001D000031DED283D103E14D52102303702031DCA
:1001E000F428BD103E14DD2103303702031DFB2827
:1001F0003D113E14E52104303702031D0229BD11D3
:100200003E14ED2111295F08F039A03C0319112992
:1002100032180D292F18112910292F1C11291029E6
:10022000F521B70A05303702031808009528013078
:10023000B600B300B400B500B70085018701B11363
:100240001A227B20B30B5229031085190314B90D10
:10025000F030390203197929B41F8501B41F8701D1
:10026000B41F8510B40B5229B50B52290230B500CA
:10027000013037020319FE2102303702031903222D
:100280000330370203190C220430370203191522F8
:100290003708B6080319B600031950298514B603A8
:1002A000FA30B400311D21293111321C5C292D098D
:1002B0000339AD00AE09AF092F1CB1132F1C212942
:1002C000B11B21292E182129B1178B132030370794
:1002D000BB002F08BA008D2110303707BB002E0855
:1002E000BA008D2100303707BB002D08BA008D21E0
:1002F0008B171E2285018701B70AB6010530370228
:10030000031C2129302208003E1C08003E1010303A
:10031000BB003D08BA008D2108008B133A088316F4
:100320001C159A003B089B0055309D00AA309D008B
:100330009C1464009C1899291C1183128B170800C7
:10034000831600309B001C141A088312DF008316EA
:1003500020309B001C141A088312C1000130C11BFD
:10036000C100C1080319C100080007128716400820
:100370004107D0000F08D10008000512871540087A
:100380004107D2000F08D300080007118516400866
:100390004107D4000F08D500080007108714400853
:1003A0004107D6000F08D70008008712071640083B
:1003B0004107D0000F08D10008008711051640083A
:1003C0004107D2000F08D300080085120715400826
:1003D0004107D4000F08D500080087100714400813
:1003E0004107D6000F08D7000800071205120711B1
:1003F0000710871287118512871008003F093039CE
:100400008700BF000800380910398500B8003F098F
:1004100008398700BF000800380920398500B80076
:100420003F0904398700BF0008003F0903398700EE
:10043000BF000800B801BF01BF160800B801BF0126
:1004400001303702031D252ABF1502303702031D74
:100450002A2AB81603303702031D2F2ABF140800BA
:1004600008005F080F390A3C03195E2A5008400251
:10047000031D402A51080F02031C402A071287124D
:1004800052084002031D4A2A53080F02031C4A2A3D
:100490000512871154084002031D542A55080F0203
:1004A000031C542A0711851256084002031D5E2AB8
:1004B00057080F02031C5E2A071087100C1C080047
:1004C0000C10C00A851008000C1C6C280C10C00B06
:0C04D0006C284108C0008501870108006D
:084000000100030005000800A7
:02400E00CC01E3
:10420000010003000300030003000200020002009B
:1042100002000000000000000000FF00FF00FF009F
:10422000000000000000000000000000000000008E
:104230000000C000C000C000C000FF00FF00FF0081
:104240000100C300F300CF00FF00C300F300CF0064
:10425000FF00C300F300CF00FF00FF00FF00FF00DE
:10426000FF00FF00FF00FF00FF00FF00FF00FF0056
:10427000FF00FF00FF00FF00FF00FF00FF00FF0046
:10428000FF00FF00FF00FF00FF00FF00FF00FF0036
:10429000FF00FF00FF00FF00FF00FF00FF00FF0026
:1042A000FF00FF00FF00FF00FF00FF00FF00FF0016
:1042B000FF00FF00FF00FF00FF00FF00FF00FF0006
:1042C000FF00FF00FF00FF00FF00FF00FF00FF00F6
:1042D000FF00FF00FF00FF00FF00FF00FF00FF00E6
:1042E000FF00FF00FF00FF00FF00FF00FF00FF00D6
:1042F000FF00FF00FF00FF00FF00FF00FF00AA001B
:00000001FF
